:103800005CC000008FC0000073C0000071C00000E9
:103810006FC000006DC000006BC0000069C00000F8
:1038200067C0000065C0000063C0000061C0000008
:103830005FC000005DC000005BC0000059C0000018
:1038400057C0000055C0000053C0000051C0000028
:103850004FC000004DC000004BC0000049C0000038
:1038600047C0000045C00000040309041C037700A2
:10387000770077002E00660069007300630068001F
:103880006C002E00640065000E03550053004200DA
:1038900061007300700012011001FF000008C016E3
:1038A000DC05020101020001090212000101008091
:1038B0003209040000000000000011241FBECFEFF9
:1038C000D4E0DEBFCDBF11E0A0E0B1E0E0EBFFE36C
:1038D00002C005900D92A630B107D9F711E0A6E01D
:1038E000B1E001C01D92AC33B107E1F771D15EC305
:1038F00087CFA82FB92F80E090E041E050EA609593
:1039000030E009C02D9182279795879510F0842784
:103910009527305EC8F36F5FA8F30895EADF8D93B3
:103920009D930895CF93CFB7CF93C3954C9BE9F761
:103930004C9B0BC04C9B09C04C9B07C04C9B05C0CB
:103940004C9B03C04C9B01C0C0C0C0911F01DF93C2
:10395000DD27CA5DDE4F2F932FEF4C9B03C02F91C5
:10396000DF91E6CF0F931F934F936F9309B104FB41
:1039700020F93F933BE05F931EC04E7F012F19B1AA
:103980001471E1F0216000001DC0102F4D7F2260F6
:10399000000009B1047191F01DC04B7F2460012F1C
:1039A000000019B1147151F01EC019B1147131F039
:1039B000477F28601BC019B1147109F462C04FEF32
:1039C000297FD9F2012704FB21F909B10471B1F370
:1039D000237FD9F2102714FB22F900C019B114710A
:1039E00069F3277ED1F2012704FB23F92F7CE9F24A
:1039F00009B1047119F3102714FB24F92F7929F167
:103A000000C019B11471E9F1012704FB25F92F73E6
:103A100011F100C009B10471A1F1102714FB26F9BE
:103A20002230F8F000C019B1147159F1012704FBDC
:103A300027F92430E0F04227000009B1499310270C
:103A400014FB20F93150C8F0B6CF4F7E09B1047194
:103A5000C1F02061D3CF206219B1147191F04F7D74
:103A6000D6CF4F7B09B1047161F02064D9CF4F7775
:103A700019B1147131F02068DCCF11E01CBB0027B4
:103A800017C03B503195C31BD04011E01CBB0881CF
:103A9000033CF9F00B34E9F020911D011981110F5D
:103AA0001213EDCF093651F10D3211F0013E39F705
:103AB000009324015F913F916F914F911F910F915E
:103AC0002F91DF91CCB3C0FD30CFCF91CFBFCF913D
:103AD000189520912401222369F3109122011123CA
:103AE00031F5343032F13093220120931E011091D0
:103AF0001F013BE0311B30931F011BC000912201CD
:103B00000130ACF40AE53091000134FD13C000939C
:103B10000001C2E1D1E012C005271127000019C041
:103B2000052711271FC005271127000024C04AE5DB
:103B300002C032ED432FC4E1D0E032E01AB114618B
:103B40005C9A0BB11AB954E120E866E020FF052722
:103B500027950BB917951C3FF8F66A95B9F720FF22
:103B60000527279500000BB917951C3FC8F620FFC5
:103B700005272795179566E01C3F0BB9A0F62991FC
:103B80003A9521F70B7E10912301110F0BB9C65105
:103B9000D04011F010931D0111E01CBB00611AB15F
:103BA0001B7E402F4B7E53E05A95F1F700C00BB9B6
:103BB0001AB94BB97FCF1BB8F8941DBA109269009F
:103BC00081E085BF15BEE0911001F09111010995CA
:103BD00088E10FB6F89480936000109260000FBEE9
:103BE0005F9A04B601FECBC114BE81E085BF82E0BE
:103BF00085BF4F99C4C1809169008260809369003C
:103C0000E89A549A20E005C0A89586EA9EE00197BC
:103C1000F1F72150C9F754987894FF2400E090916F
:103C20002201935097FD2EC180911F01CCE0D0E07E
:103C3000C81BD109CA5DDE4F80911E018D3209F08B
:103C4000C4C0983009F01CC183EC809312018AE54E
:103C50008093000110920A013881832F8076298198
:103C6000882309F443C086E091E09093210180937A
:103C700020012330C9F49B818C812A81203339F4BF
:103C80008370E82FF0E0EE5FFE4F808109C0203A9C
:103C900011F476D105C0203C11F46D8179D180E01A
:103CA0008093090194E087C0253011F491E083C02E
:103CB000822F8450863098F48A819B8190930D01E5
:103CC00080930C01293081F09E8190930E018D81AB
:103CD000827080930F0137FD69C02FEF68C02230DA
:103CE00019F481E080930B0190E065C08A81109205
:103CF0001B01222331F410921C012BE131E092E0F0
:103D000050C0253019F48093230148C02630B1F506
:103D10008B81813019F486E998E304C0823041F444
:103D200088EA98E3909321018093200192E122C0D8
:103D30008330F9F48A81882341F488E698E39093EC
:103D400021018093200194E015C0813041F48CE67C
:103D500098E390932101809320019CE10BC0823075
:103D600041F488E898E390932101809320019EE03C
:103D700001C090E080E480930A011DC0283019F44E
:103D800025E231E009C0293019F48093250106C0ED
:103D90002A3021F42BE131E091E003C02BE131E046
:103DA00090E0309321012093200105C0292F80E865
:103DB00080930A0107C08F81882319F42E81291767
:103DC00008F0292F209301015BC080910A0187FF31
:103DD00057C080910E01592F891708F4582F851B61
:103DE00080930E0160E0882309F461E070910F0177
:103DF000E0910C01F0910D0140E037C0CF018F77C9
:103E00009070892B49F4F89483E080935700E895EB
:103E1000789407B600FCFDCF4E5FF8948991999194
:103E200021E00C0120935700E895112478949F011C
:103E30002E5F3F4FC9018F779070892B31F0662339
:103E400099F0451788F0772379F0F89485E080930E
:103E50005700E895789407B600FCFDCFF89481E10F
:103E600080935700E8957894F901451708F4C6CF78
:103E7000F0930D01E0930C01662311F01092010103
:103E8000109222018091000184FF65C080910101A0
:103E90008F3F09F460C0182F893008F018E0811BAB
:103EA000809301018091120198E889278093120183
:103EB000112309F43EC080910A0187FF1EC0809142
:103EC0000E01811708F4182F811B80930E01E091D9
:103ED0000C01F0910D01A3E1B1E003C084918D9339
:103EE0003196812F90E08D5E9E4FA817B907B1F7EC
:103EF000F0930D01E0930C011AC0E0912001F091C4
:103F0000210186FF09C0912FA3E1B1E084918D9337
:103F100031969150D9F707C0912FA3E1B1E081917B
:103F20008D939150E1F7F0932101E0932001193036
:103F300060F483E191E0612FF1DC612F6C5F6C3004
:103F400041F08FEF8093010104C08FEF8093010156
:103F50006EE16093000194E189B1847131F4915074
:103F6000D9F71092230110921D0180910B01882333
:103F700021F0FA9411F4015011F04F9B50CE1BDE4A
:103F8000F999FECF92BD81BDF89A992780B5089521
:103F9000262FF999FECF1FBA92BD81BD20BD0FB665
:103FA000F894FA9AF99A0FBE01960895F894FFCF03
:063FB0005AFF1E940600FA
:0400000300003800C1
:00000001FF
